S10500000152A7
S1050008027F71
S1090100000406800A025F
S105010C4000AD
S11B01150002D20347038103E80000013E013E013E013E01520E330EA3
S114012D330E330E33200006320632063206320E33C7
S11B01521A5086011F8B10CE0100860AB720124FB72021B7202386ECEB
S11B016AB7204C86C0B7204B86F0B7204FB7204386BFB72040B72042C3
S11B0182867FB7204EB7204D86EEB7204CBD05F88640970CC660B6205D
S11B019A402BFBB620402AFB5A26F34F970F43B72805B728068605B7F2
S11B01B2201286C0B7201086820D0D2712C60153F728068E0439BF01AD
S11B01CA1CC601D7158A01970F43B72807BD04F71CEF108E0120BD05AC
S11B01E29126531F89BD05919711BD059181C0263C96115A260497029A
S11B01FA202E5A2604970320355A2604970420205A2604970520195A16
S11B02122609910D2705970D7E01525A2618847F9701961184809700ED
S11B022ABD05F82009BD0591260481C026F7B6201281052719108E01AD
S11B024234AE24AC26270F1A10B6201281052704AD9F01181CEF0D153D
S11B025A2F20108E012AAE24AC2627161A100D152F0E108E012AAE246B
S11B0272AC262704AD9F011C1CEF7E01DCB620112A1585082709AD9F75
S11B028A0116B620112A0885102704AD9F0118B62803438501260484AB
S11B02A206271D971085C42706AD9F011A961085322706AD9F011C96E9
S11B02BA1085082703BD04F7B6204D2A03BD05483B108E0116BD058C11
S11B02D2F6201085072639C1C02635108E0116BD058CF6201085072648
S11B02EAE05D2725C10026033F20D612C1C027181F98108E0120BD0546
S11B0302A026C6108E0116BD058C108E0120200C39108E0116BD058C29
S11B031A108E012AF62010850726111F98BD05A0260A81C026E2AE22B3
S11B0332AF2420A7AE24AF2281C0268D209D108E0118BD058C108E011D
S11B034A34BD05912604B72010398609B72012108E0118BD058C108EAB
S11B03620134BD059126A9C605F72012B7201020CD960F847F43B72896
S11B037A07960F43B72807108E0134AE24AF224FBD05A0108E011ABDF5
S11B0392058C8504272F108E0134B628044381C0270881DB260FC6DD43
S11B03AA2002C6DC86DBBD05A026BE1F98BD05A026B7961085802609FC
S11B03C2854026BB39858027B6108E0134BD05BC26AD86C0BD05A0266C
S11B03DAA6AE22AF2420A8108E011CBD058C86FF97150D0D2636960FA1
S11B03F2847F970F9E06272C4F43B728038643BD0565DC068E041FBD9B
S11B040A0574108E011CBD058C85021027008F4F43B72803398E0426A2
S11B0422BF011C39108E012ABD059143B728030D0D2634866320228643
S11B043AFF9715960F8A40970F43B7280720548673206ABD059126F756
S11B045281C027F7B728038673BD0565108E011CBD058C8520273F8693
S11B046A43BD0565108E011CBD058C108E012ABD0591263781DB2613F5
S11B0482BD05911F8986C0C1DC270C86DBC1DD27061F9881C027B4430B
S11B049AB72803108E011CBD058C851027CD108E012ABD05912604810B
S11B04B2C026F78653BD0565108E011CBD058CDC0A27138E04D8BD05FC
S11B04CA74108E011CBD058C4F43B7280339860197150D0D2614960FC0
S11B04E284BE8A80970F43B728070F158640970C8D037E03E1B6280284
S11B04FA0D0D2623438440910C271C970C27190D152B140F158620B7D7
S11B0512204EFC2048960F8A80970F43B7280739960F847F970F43B7FC
S11B052A2807BD03730D1526EE2007BD05EED1032307DC088E0535207C
S11B0542318601971539FC20480D14270A0A144D26015CFD2048398638
S11B055A20B7204EB620486E9F011E9713960F84CF9A13970F43B728DF
S11B05720739BF011E97144F5D26060A142BD84353FD204886A0B720B3
S11B058A4E393510AFA439AE26AC242719A6848D18AF261A0439AE224E
S11B05A21F138D0DAC262706A7C4AF2220ED1CFB393001AC282602AEFE
S11B05BAA439AE22AC2427EE8D0A26F58D0626F1AF2220CF8D1026E9CB
S11B05D28D0C26E5A68481DB27C18DD520BDACA42602AE28301FAC244F
S11B05EA26B120C28615D60E3DCB35D70E39C6240D00270158D711966D
S11B0602023DDD06D61196043DDD08D61196053DDD0A0D0126048604AF
S11B061A9701C6604F4CD0012EFB0D0026014480022B045FFD2044394F
S9030000FC
